:100000000C9450000C946D000C946D000C946D00D9
:100010000C946D000C946D000C946D000C946D00AC
:100020000C946D000C946D000C9409060C946D00FA
:100030000C946D000C9440060C9489060C946D0091
:100040000C946D000C946D000C946D000C946D007C
:100050000C946D00342E332E34002C206176722DDA
:100060006763633A2000312E362E38002C206176EB
:10007000722D6C6962633A2000312E322E3020627C
:1000800075696C643A323031303033303600686F25
:100090006E64612D7274702C207665722E200000C3
:1000A00011241FBECFE5D8E0DEBFCDBF11E0A0E632
:1000B000B0E0E4ECFBE102C005900D92A836B10778
:1000C000D9F712E0A8E6B1E001C01D92AE3DB1073C
:1000D000E1F70E94F3030C94E00D0C940000DC01A6
:1000E00010926F0110926E0110926D0161157105F1
:1000F00099F040E020E030E0FD01E20FF31F808145
:10010000480F2F5F3F4F26173707B0F370936E01EC
:1001100060936D0140936F0180916F01089588EDA8
:1001200091E064E070E041E050E00E94140708951F
:1001300088ED91E061E070E045E050E00E94140736
:10014000882329F09091D801809170019813089527
:1001500081E08093D90188E28093DA0181E3809382
:10016000DB0189ED91E063E070E00E949E07089555
:100170002FE32093D80120936F0181E090E09093CA
:100180006E0180936D012093D90188ED91E062E0CA
:1001900070E00E949E070895809169018823A1F470
:1001A00022E42093D80120936F0181E090E09093A6
:1001B0006E0180936D012093D90188ED91E062E09A
:1001C00070E00E949E0708952FE4EBCF1092690122
:1001D000809170018093D80189ED91E063E070E037
:1001E00045E050E00E9414078823E1F18091D90195
:1001F0008823C9F580E091E061E071E0909372019D
:10020000809371018CED91E045E050E00E9414076D
:10021000882341F16091710170917201DB011496A4
:1002200010926F0110926E0110926D01109799F06B
:1002300090E020E030E0F901E852FE4F8081980F15
:100240002F5F3F4F2A173B07B0F3B0936E01A09387
:100250006D0190936F01A852BE4F9C9180916F01E8
:10026000981731F0089590E0BC016F5F7F4FC6CFC3
:100270009091DA0180E02091DB01820F911D4CED1D
:1002800051E00E94CC04882341F59091DA0180E08E
:100290002091DB016091710170917201820F911DBB
:1002A0004CED51E00E94CC048823B9F49091DA011E
:1002B00080E02091DB016091710170917201820FE9
:1002C000911D4CED51E00E94CC04882331F40E9432
:1002D000260481E080936901089510926C011092C8
:1002E0006B018091710190917201009791F0E8ED9E
:1002F000F1E020E030E0AC014E0F5F1F8481280F59
:10030000311D3196E417F507C9F730936C0120933E
:100310006B0180916B0190916C018093D801909357
:10032000D90188ED91E062E070E00E949E07CFCF96
:1003300010926901809170018093D80189ED91E05C
:1003400063E070E045E050E00E941407882309F460
:1003500043C080916801882309F43FC08091D9018E
:1003600090E0019690937201809371016091710108
:10037000709172016F5F7F4F8CED91E045E050E02E
:100380000E941407882341F16091710170917201FC
:10039000DB01149610926F0110926E0110926D01A4
:1003A000109799F090E020E030E0F901E852FE4F1C
:1003B0008081980F2F5F3F4F2A173B07B0F3B09310
:1003C0006E01A0936D0190936F01A852BE4F9C9156
:1003D00080916F01981751F008958091D901882379
:1003E00011F090E0BFCF80E091E0BCCF9091DA01B6
:1003F00080E02091DB01820F911D4CED51E00E94C5
:10040000CC04882341F59091DA0180E02091DB0152
:100410006091710170917201820F911D4CED51E05C
:100420000E94CC048823B9F49091DA0180E02091F5
:10043000DB016091710170917201820F911D4CED91
:1004400051E00E94CC04882331F40E94260481E00C
:100450008093690108958FE40E94EE07F6CF8091A2
:1004600070018093D80189ED91E062E070E045E091
:1004700050E00E9414078823A1F04091D901809197
:10048000D801840F22E030E030936E0120936D019B
:1004900080936F019091DA01981721F086E40E9411
:1004A000EE07089510926801442319F081E08093CB
:1004B00068018FE40E94EE0708951092690188EDAB
:1004C00091E062E070E045E050E00E94140788236C
:1004D00009F408959091D80180E02091D901820F0C
:1004E000911D0E946004FC0180818093DA010E94CA
:1004F000EE070E94260481E080936901089510921E
:100500006901809170018093D80189ED91E064E0E8
:1005100070E045E050E00E9414078823C9F0E8ED40
:10052000F1E020E08191280F81E0EC3DF807D1F760
:1005300084E090E090936E0180936D0120936F01B1
:100540008081821731F00E94260481E08093690146
:1005500008956091D901662309F043C060E071E01D
:1005600070937201609371019091DA0180E02091A3
:10057000DB01820F911D48ED51E00E9470046091F3
:1005800071017091720110926F0110926E011092C0
:100590006D016115710599F090E020E030E0F901FE
:1005A000E852FE4F8081980F2F5F3F4F2617370785
:1005B000B0F370936E0160936D0190936F01FB0136
:1005C000E852FE4F80916F0180836F5F7F4F88ED0F
:1005D00091E00E949E070E94260481E080936901B9
:1005E000B7CF70E0BDCF809170018093D80189EDC5
:1005F00091E066E070E045E050E00E941407882337
:10060000B9F0E8EDF1E020E08191280F41E0EE3D06
:10061000F407D1F786E090E090936E0180936D012E
:1006200020936F018081821721F086E40E94EE07FB
:1006300008958FE40E94EE0780E090E000000196AC
:100640005FEF8F3F9507D1F79091D90180E020911E
:10065000DA01AC01420F511D9A0160E08091DB018B
:10066000811161E040E08091DC01811141E0C9012C
:100670002091DD010E948608089588ED91E061E0F7
:1006800070E045E050E00E941407882329F0909123
:10069000D80180917001981308958EE890E00E942F
:1006A0005D0889E790E00E945D088CE690E00E947A
:1006B0005D0886E690E00E945D088AE590E00E9471
:1006C0005D0884E590E00E945D0808958AE691E067
:1006D0000E94C006982F8093700180916A01882340
:1006E00071F0933561F1943558F09835D1F1993521
:1006F000C0F4963569F19735C1F00E94B8000895AD
:10070000963461F19734A0F49234F9F09534A9F756
:1007100088ED91E064E070E041E050E00E94140751
:100720000895923779F0973741F70E94980108951C
:100730009D3489F0923509F70E947F0208950E9446
:10074000CC0008950E945D0208950E942F02089532
:100750000E94980008950E94F30208950E943D03AC
:1007600008950E94E60008958FEF8ABB84BBB89A73
:10077000B99ABA9ABB9ABC9A8A9A8B9A8C9A8D9A91
:100780008E9A8F9A939894981BBA15BA929AC09A97
:10079000959A969AC49AC19AC39AC29A979880B722
:1007A000846080BF089582B390E1892782BB089559
:1007B000089508950E946F07882311F00E94660330
:1007C0000E94260481E08093690108950E94B40389
:1007D0000E94360680EF93E260E041E021E00E9453
:1007E000860878940895FF920F931F930E94E60362
:1007F0000E940E05882339F4949A80E090E01F91BE
:100800000F91FF9008950E94D9058823A9F3939A28
:1008100081E0809369010E94260410E000E080E1FD
:10082000F82E02C00E94DA030E942E068823D1F31C
:100830001F5F1A30B9F70F5F0A3011F010E0F2CFE6
:1008400082B38F2582BB10E000E0ECCF8091730172
:10085000882361F49298C09A959A969AC49AC198FE
:10086000C398C29A979881E080937301089510927B
:1008700073019298C09A959A969AC498C19AC39A0D
:10088000C298979814BA15BA00000895109273018F
:10089000929AC09A959A969AC498C19AC39AC29805
:1008A000979A8FEF84BB000008958BBB969A000047
:1008B000969800009BBB959A0000959800000895BB
:1008C0000F931F938C010E943704C8010E945504A6
:1008D00083B38093760186E791E01F910F9108958D
:1008E000CF92DF92EF92FF920F931F93CF93DF93FC
:1008F0006C018B017A0110927501109274016115DF
:100900007105A9F0C0E0D0E0CE018C0D9D1D0E94C4
:100910006004FC01D701AC0FBD1F80818C93219630
:10092000C017D10788F31093750100937401C701B4
:10093000DF91CF911F910F91FF90EF90DF90CF90BB
:1009400008950F931F93CF93DF93EC01062F10E0D0
:100950000E944604CE010E94550405BBC0980000C9
:10096000C09ACE010E946004FC01E0810E1761F084
:100970001F5F133069F7E0937701939880E0DF9170
:10098000CF911F910F9108950093770181E0DF913E
:10099000CF911F910F910895AF92BF92CF92DF92A6
:1009A000EF92FF920F931F93CF93DF935C016B0144
:1009B00010927501109274016115710519F17A0197
:1009C000C0E0D0E000E010E00AC08E010F5F1F4FD2
:1009D0000894E11CF11C0C151D0580F4E801CE0102
:1009E0008A0D9B1DF70160810E94A104882369F78D
:1009F000109375010093740180E005C01093750198
:100A00000093740181E0DF91CF911F910F91FF90CE
:100A1000EF90DF90CF90BF90AF900895FF920F932B
:100A20001F93CF93DF9310927801C0E0D0E0CE0106
:100A300060E00E94A1042196D7FFF9CF10927501C2
:100A400010927401C0E0D0E000E010E001C0E801C5
:100A5000CE010E946004FC018081882391F58E0103
:100A60000F5F1F4F17FFF3CF1092750110927401A3
:100A7000C0E0D0E000E010E00EC035E5F32ECE017E
:100A80006F2D0E94A104882381F08E010F5F1F4FFC
:100A900017FD22C0E801C0FFF0CF2AEAF22ECE01F6
:100AA0006F2D0E94A104882381F7F09278011093A2
:100AB000750100937401DF91CF911F910F91FF9009
:100AC0000895109375010093740180E0DF91CF9138
:100AD0001F910F91FF900895F09278011092750187
:100AE00010927401C0E0D0E000E010E008C0E535ED
:100AF00079F48E010F5F1F4F17FD17C0E801CE017B
:100B00000E946004FC01E081C0FFF1CFEA3A89F362
:100B10001093750100937401E093780180E0DF91F8
:100B2000CF911F910F91FF900895E093780110925B
:100B3000750110927401C0E0D0E000E010E00FC039
:100B40009AEAF92ECE016F2D0E94A104882309F4A0
:100B5000ACCF8E010F5F1F4F17FD06C0E801C0FF2D
:100B6000EFCF85E5F82EEECFF09278011092750167
:100B700010927401C0E0D0E000E010E008C0EA3A52
:100B800039F68E010F5F1F4F17FD0BC0E801CE0134
:100B90000E946004FC01E081C0FFF1CFE53589F3DC
:100BA000B7CF1093750100937401E093780181E051
:100BB0008DCF0F931F93CF93DF938FEF80937801A7
:100BC0001092750110927401C0E0D0E000E010E0D6
:100BD00001C0E801CE016FEF0E94A104882379F0E3
:100BE0008E010F5F1F4F17FFF4CF10937501009315
:100BF000740181E0DF91CF911F910F9108951093BF
:100C000075010093740180E0DF91CF911F910F91E6
:100C100008951F920F920FB60F9211248F939F93F6
:100C200080917A018F5F80937A0180917A01893077
:100C300071F410927A0181E08093790180917B01B7
:100C400090917C01019690937C0180937B019F9110
:100C50008F910F900FBE0F901F9018958091790182
:100C6000882319F01092790181E008958FEF8CBFED
:100C700082E089BF88E083BF83B7836083BF089524
:100C80001F920F920FB60F9211248F939F93EF93A1
:100C9000FF935C9B05C08091D70180618093D70151
:100CA0005B9B05C08091D70188608093D7015A9BD8
:100CB00005C08091D70184608093D7018091D701CE
:100CC00081FF06C08091D4018F5F8F738093D40120
:100CD000E091D301F0E08CB1ED57FE4F808380911D
:100CE000D3018F5F8F738093D3019091D301809153
:100CF000D401981729F48091D70182608093D7019D
:100D0000FF91EF919F918F910F900FBE0F901F90C9
:100D100018951F920F920FB60F9211248F939F93E5
:100D2000EF93FF939091D6018091D5019817D9F058
:100D3000E091D601F0E0ED53FE4F80818CB98091B7
:100D4000D6018F5F8F708093D6018091D7018E7FFF
:100D50008093D701FF91EF919F918F910F900FBEDC
:100D60000F901F9018958091D70180FDE1CF559885
:100D7000F1CF8091D70190E0969587958170089585
:100D8000DC018091D70181FD13C09091D301809146
:100D9000D4018917C0F59091D3018091D401981B9B
:100DA000992331F4109709F01C92E0E08E2F0895FA
:100DB000E091D401F0E0ED57FE4FE081E093810136
:100DC0008091D4018F5F8F738093D4018091D7017C
:100DD0008D7F8093D701109749F38091D7018C7153
:100DE000F9F01C928091D7018F7E8093D70180917A
:100DF000D7018B7F8093D7018091D701877F809324
:100E0000D7018E2F08959091D3018091D401981726
:100E100048F69091D3018091D401905C981BC0CF8B
:100E200081E08C938E2F0895CF92DF92EF92FF9204
:100E30000F931F93CF93DF937C016B01EA01611540
:100E4000710509F44AC000E010E010927C01109294
:100E50007B018091D70181FF13C082E891E00E945D
:100E6000C006F7018083809182018823F9F00F5F2B
:100E70001F4F0C151D0588F50894E11CF11CE5CFEA
:100E80009091D3018091D4018917D0F49091D3012E
:100E90008091D401981B992301F72097F1F280915A
:100EA0007B0190917C018C179D0799F680E0DF9182
:100EB000CF911F910F91FF90EF90DF90CF90089509
:100EC0009091D3018091D401981738F79091D30174
:100ED0008091D401905C981BDECF81E0E8CF8091B7
:100EE000D70181FD1BC09091D3018091D401891756
:100EF00070F09091D3018091D401981790F4909163
:100F0000D3018091D401905C981B892F0895909112
:100F1000D3018091D401981B892F089590E4892FE3
:100F2000089590E0892F08958091D3018093D40192
:100F30008091D7018D7F8093D7010895DC016115E1
:100F40007105A9F586E091E09093800180937F017F
:100F500066E071E020E030E09C918091D70180FD57
:100F6000FCCFE091D501F0E0ED53FE4F90838091EE
:100F7000D5018F5F8F708093D5019091D5018091BD
:100F8000D601981741F0559A2F5F3F4F2617370724
:100F900068F41196E1CF8091D70181608093D701E9
:100FA000559A2F5F3F4F2617370798F3089581E032
:100FB0006730780740F47093800160937F0161157A
:100FC000710541F6089566E071E0709380016093C9
:100FD0007F016115710509F0BDCFF4CF982F809185
:100FE000D70180FDFCCFE091D501F0E0ED53FE4F3D
:100FF00090838091D5018F5F8F708093D501909100
:10100000D5018091D601981729F48091D70181608C
:101010008093D701559A0895DC0161157105A9F5F2
:1010200086E091E090937E0180937D0166E071E01F
:101030009C91992309F440C020E030E08091D701D1
:1010400080FDFCCFE091D501F0E0ED53FE4F9083A1
:101050008091D5018F5F8F708093D5019091D501DC
:101060008091D601981759F0559A2F5F3F4F261758
:10107000370720F411969C91992301F708958091E8
:10108000D70181608093D701EFCF81E06730780787
:1010900040F470937E0160937D016115710541F606
:1010A000089566E071E070937E0160937D016115A3
:1010B000710509F0BDCFF4CF08959C01FC01949116
:1010C0009923E9F08091D70180FDFCCFE091D50113
:1010D000F0E0ED53FE4F90838091D5018F5F8F70CC
:1010E0008093D5019091D5018091D601981741F058
:1010F000559A2F5F3F4FF9019491992319F708955D
:101100008091D70181608093D701F2CF0F931F9315
:10111000042F122F1092D3011092D4011092D501F6
:101120001092D6011092D701662389F1BC0180E0AC
:1011300090E00E94390B9B01AC0160E070E080E917
:1011400096E40E948D0A20E030E040E85FE30E94D0
:101150002F0A0E947D0D962F82E28BB970BD99B93E
:1011600088E98AB9002351F08EE0113051F0123035
:1011700039F1806880BD1F910F91089586E011308C
:10118000B1F78062806880BD1F910F910895BC0106
:1011900080E090E00E94390B9B01AC0160E070E0C0
:1011A00080E196E40E948D0A20E030E040E85FE3B1
:1011B0000E942F0A0E947D0D962F80E28BB9CECF20
:1011C0008063806880BD1F910F910895A0E0B0E01A
:1011D000ECEEF8E00C94460DDC012B01FA019C9139
:1011E000923008F436C1EB018881823008F430C1B6
:1011F000943061F4843009F02CC1FD019181898122
:10120000981709F426C1A0E6B0E023C1843009F4A0
:101210001FC18230A9F4923009F01BC19A01AD01BF
:1012200088E0EA010990AE01E90109929E0181502E
:10123000C1F7E2018981ED0199818923818306C18A
:10124000923009F405C1ED012A803B80EB018A81CF
:101250009B81ED01AC80BD80CE80DF80EB01EC8016
:10126000FD800E811F819101281B390BB90137FFC9
:1012700004C066277727621B730B603271050CF080
:1012800061C0121613066CF537014801062E04C022
:1012900096948794779467940A94D2F721E030E08B
:1012A00040E050E004C0220F331F441F551F6A95D1
:1012B000D2F721503040404050402E213F21402362
:1012C0005123211531054105510521F021E030E080
:1012D00040E050E079018A01E628F7280829192919
:1012E0003CC0232BD1F1260E371E35014601062EB8
:1012F00004C096948794779467940A94D2F721E077
:1013000030E040E050E004C0220F331F441F551F5F
:101310006A95D2F721503040404050402A213B216D
:101320004C215D21211531054105510521F021E0B8
:1013300030E040E050E059016A01A628B728C828EB
:10134000D9280BC0821593052CF01C01AA24BB24BC
:10135000650103C0EE24FF248701ED019981E201BC
:101360008981981709F445C0992339F0A80197019C
:101370002A193B094C095D0906C0A60195012E19E1
:101380003F09400B510B57FD08C011823382228266
:1013900024833583468357831DC081E08183338254
:1013A000228288279927DC01821B930BA40BB50BA3
:1013B00084839583A683B7830DC0220F331F441FF8
:1013C000551F2483358346835783828193810197F8
:1013D000938382832481358146815781DA01C90153
:1013E0000197A109B1098F5F9F4FAF4FBF4328F30A
:1013F0000BC0918333822282EA0CFB1C0C1D1D1D45
:10140000E482F5820683178383E08083248135811B
:101410004681578157FF1AC0C901AA2797FDA09599
:10142000BA2F81709070A070B0705695479537951F
:101430002795822B932BA42BB52B84839583A6838E
:10144000B78382819381019693838283DF0101C0F8
:10145000D201CD01CDB7DEB7E2E10C94620DA0E27E
:10146000B0E0E5E3FAE00C94520D69837A838B8354
:101470009C832D833E834F835887E9E0EE2EF12C29
:10148000EC0EFD1ECE010196B7010E94D60C8E0116
:101490000F5E1F4FCE010596B8010E94D60C8A89B7
:1014A00091E089278A8BC701B801AE01475E5F4F83
:1014B0000E94E6080E94010CA096E6E00C946E0DD6
:1014C000A0E2B0E0E6E6FAE00C94520D69837A837C
:1014D0008B839C832D833E834F835887F9E0EF2EC7
:1014E000F12CEC0EFD1ECE010196B7010E94D60C28
:1014F0008E010F5E1F4FCE010596B8010E94D60CDB
:10150000C701B801AE01475E5F4F0E94E6080E9426
:10151000010CA096E6E00C946E0DA8E1B0E0E3E9C2
:10152000FAE00C944E0D69837A838B839C832D8320
:101530003E834F835887B9E0EB2EF12CEC0EFD1E55
:10154000CE010196B7010E94D60C8E010F5E1F4F8F
:10155000CE010596B8010E94D60C2985223008F4E8
:101560007EC03989323010F4B8017CC08A859A89EE
:1015700089278A87243011F0223031F4231709F0AB
:101580006EC060E670E06EC0343039F41D861E8691
:101590001F86188A1C861B8604C0323021F484E022
:1015A0008987B7015FC02B853C858B899C89281B67
:1015B000390B3C872B87ED84FE840F851889AD8815
:1015C000BE88CF88D88CEA14FB040C051D0540F4B6
:1015D000EE0CFF1C001F111F215030403C872B8751
:1015E00020E030E040E050E080E090E0A0E0B0E4B7
:1015F00060E070E0EA14FB040C051D0540F0282BA8
:10160000392B4A2B5B2BEA18FB080C091D09B695F0
:10161000A79597958795EE0CFF1C001F111F6F5F14
:101620007F4F6F31710531F7DA01C9018F77907003
:10163000A070B07080349105A105B10561F427FD5B
:101640000AC0E114F1040105110529F0205C3F4FA7
:101650004F4F5F4F20782D873E874F87588BBE01B5
:10166000675F7F4FCB010E94010C6896EAE00C9403
:101670006A0DA8E0B0E0EFE3FBE00C944E0D7B01B7
:101680008C01611571058105910519F482E089834A
:1016900060C083E089838EE1C82ED12CDC82CB82AE
:1016A000ED82FE820F831887C801B7010E94B20B3A
:1016B000FC013197F7FF3BC0222733272E1B3F0B3E
:1016C00057016801022E04C0D694C794B794A7941A
:1016D0000A94D2F740E050E060E070E081E090E0F2
:1016E000A0E0B0E004C0880F991FAA1FBB1F2A9575
:1016F000D2F70197A109B1098E219F21A023B1231F
:101700000097A105B10521F041E050E060E070E0F4
:101710004A295B296C297D294D835E836F837887F5
:101720008EE190E08E1B9F0B9C838B8312C03097C1
:1017300081F00E2E04C0EE0CFF1C001F111F0A9436
:10174000D2F7ED82FE820F831887CE1ADF0ADC8281
:10175000CB821A82CE0101960E94010C2896EAE003
:101760000C946A0DEF92FF920F931F937B018C01F3
:1017700080E0E81680E0F80681E0080780E01807BE
:1017800088F48FEFE816F1040105110531F028F017
:1017900088E090E0A0E0B0E017C080E090E0A0E03A
:1017A000B0E012C080E0E81680E0F80680E00807AC
:1017B00081E0180728F088E190E0A0E0B0E004C0E4
:1017C00080E190E0A0E0B0E020E230E040E050E0D6
:1017D000281B390B4A0B5B0B04C016950795F79431
:1017E000E7948A95D2F7F701E859FF4F8081281BCB
:1017F000310941095109C9011F910F91FF90EF90E3
:101800000895DF92EF92FF920F931F93FC01E48003
:10181000F58006811781D1808081823048F480E094
:1018200090E0A0E1B0E0E82AF92A0A2B1B2BA5C022
:10183000843009F49FC0823021F4EE24FF24870114
:1018400005C0E114F1040105110519F4E0E0F0E030
:1018500096C0628173819FEF623879070CF05BC09C
:1018600022E83FEF261B370B2A3131052CF020E010
:1018700030E040E050E02AC0B801A701022E04C0C9
:1018800076956795579547950A94D2F781E090E051
:10189000A0E0B0E004C0880F991FAA1FBB1F2A95C3
:1018A000D2F70197A109B1098E219F21A023B1236D
:1018B0000097A105B10521F081E090E0A0E0B0E043
:1018C0009A01AB01282B392B4A2B5B2BDA01C9017A
:1018D0008F779070A070B07080349105A105B1052C
:1018E00039F427FF09C0205C3F4F4F4F5F4F04C0C2
:1018F000215C3F4F4F4F5F4FE0E0F0E02030A0E031
:101900003A07A0E04A07A0E45A0710F0E1E0F0E04F
:1019100079018A0127C06038710564F5FB01E1583F
:10192000FF4FD801C7018F779070A070B0708034DE
:101930009105A105B10539F4E7FE0DC080E490E002
:10194000A0E0B0E004C08FE390E0A0E0B0E0E80EDB
:10195000F91E0A1F1B1F17FF05C016950795F79460
:10196000E794319687E016950795F794E7948A9562
:10197000D1F705C0EE24FF248701EFEFF0E06E2FD2
:10198000679566276795902F9F77D794DD24D79426
:101990008E2F8695492F462B582F5D29B701CA01F6
:1019A0001F910F91FF90EF90DF900895FC01DB01F4
:1019B000408151812281622F6F7770E0221F2227A0
:1019C000221F9381892F880F822B282F30E0991FA7
:1019D0009927991FFD0191832115310581F5411545
:1019E00051056105710511F482E032C082E89FEF74
:1019F000FD01938382839A01AB0167E0220F331FBD
:101A0000441F551F6A95D1F783E08C930AC0220FBB
:101A1000331F441F551FFD018281938101979383DA
:101A200082832030F0E03F07F0E04F07F0E45F07EB
:101A300070F3FD01248335834683578308952F3F38
:101A4000310581F4411551056105710519F484E0F2
:101A50008C93089564FF03C081E08C9301C01C92B5
:101A6000FD010FC02F573040FD013383228383E0F7
:101A70008C9387E0440F551F661F771F8A95D1F717
:101A80007064448355836683778308952F923F92D1
:101A90004F925F926F927F928F929F92AF92BF927E
:101AA000CF92DF92EF92FF920F931F93CF93DF932A
:101AB000CDB7DEB7CA1BDB0B0FB6F894DEBF0FBE87
:101AC000CDBF09942A88398848885F846E847D84D4
:101AD0008C849B84AA84B984C884DF80EE80FD80D6
:101AE0000C811B81AA81B981CE0FD11D0FB6F8944C
:101AF000DEBF0FBECDBFED01089541D0A8F19E57C6
:101B0000A8F1985160F039F1983070F5092E9927B5
:101B1000660F771F881F991F0A94D1F71CC0BB2737
:101B2000993F4CF4B111B1E0B62B672F782F88277D
:101B3000985FB1F708C0869577956795B79508F4D3
:101B4000B1609395C1F7BB0F30F411F460FF03C08F
:101B50006F5F7F4F8F4F3EF49095809570956195A4
:101B60007F4F8F4F9F4F0895689424C022C057FD28
:101B70009058440F551F59F05F3F71F04795880FFB
:101B800097FB991F61F09F3F79F087950895121692
:101B900013061406551FF2CF4695F1DF08C016163E
:101BA00017061806991FF1CF8695710561050894EF
:101BB0000895E894BB2766277727CB0197F9089506
:041BC000F894FFCFC7
:101BC4000000000000000000000102020303030300
:101BD40004040404040404040505050505050505B9
:101BE4000505050505050505060606060606060699
:101BF4000606060606060606060606060606060681
:101C04000606060606060606070707070707070768
:101C14000707070707070707070707070707070750
:101C24000707070707070707070707070707070740
:101C34000707070707070707070707070707070730
:101C44000707070707070707080808080808080818
:101C54000808080808080808080808080808080800
:101C640008080808080808080808080808080808F0
:101C740008080808080808080808080808080808E0
:101C840008080808080808080808080808080808D0
:101C940008080808080808080808080808080808C0
:101CA40008080808080808080808080808080808B0
:101CB40008080808080808080808080808080808A0
:081CC4000808080808080808D8
:00000001FF
